:040000000209793246
:01000B0032C2
:0100130032BA
:01001B0032B2
:0100230032AA
:01002B0032A2
:100979007581071208EDE582600302003302003336
:100033001207A080FEC2A7C2A7C2A7D2A7227A3204
:100043007B001ABAFF011BEA4B70F722AA82AB832B
:100053007C007D00C3EC9AED64808BF063F08095A7
:10006300F0501AC002C003C004C005120041D005FD
:10007300D004D003D0020CBC00DA0D80D7227A0161
:100083007B001ABAFF011BEA4B70F7223098FDC2BE
:10009300988599821200A7859982223098FDC2988B
:1000A30085998222AA823099FDC2998A9922AA82CD
:1000B300AB83ACF07D008D060DEE2AF582E43BF5B3
:1000C300838CF0120951FE8E07BE000280178F82C7
:1000D300C002C003C004C0051200A7D005D004D0DD
:1000E30003D00280D1227A287B087C028A828B8308
:1000F3008CF01200B122AA37BA0D127AEB7B077C7F
:10010300028A828B838CF01200B11200E9227A00FA
:100113007B008A04BC0A02802E758211C002C003D0
:100123001200A7D003D002C002C00312008FAC821A
:10013300D003D0028C028A04BC0D027A0AEB24425B
:10014300A8E0A6020B80CB1BEB2442A8E076007A42
:10015300007B007C00EC2442F88605BD000280375A
:10016300E4F54F754E0A8A828B83C002C003C00434
:10017300C0051208CEAE82AF83D005D004D003D021
:1001830002ED3395E0F8ED2EFEE83FFFEE24D0FAC2
:10019300EF34FFFB0C80BE8A828B832230980912D6
:1001A300008FAA828A3780037537FF227A2D7B0856
:1001B3007C028A828B838CF01200B11200E922AA9E
:1001C30082C374099A400F74302AFB8B82C00212D7
:1001D30000A7D002800974372AFA8A821200A72264
:1001E300AA8274F05AFBC4540FFB8B82C002C00373
:1001F3001201C2D003D002740F5AFB8B821201C2C8
:1002030022AA82AB838B047D008C82C002C00312BE
:1002130001E3D003D0028A821201E322AA82AB83D4
:10022300754E10754F278A828B83C002C003120854
:100233008FAC82AD83D003D00274302CFCE43DFD3F
:100243008C48754E10754F278A828B831208F1AA4A
:1002530082AB83754EE8754F038A828B83C002C0DD
:100263000312088FAC82AD83D003D00274302CFC10
:10027300E43DFD8C49754EE8754F038A828B83C03C
:1002830002C0031208F1AC82AD83D003D0028C020A
:100293008D03E4F54F754E648A828B83C002C003DD
:1002A30012088FAC82AD83D003D00274302CFCE4EF
:1002B3003DFD8C4AE4F54F754E648A828B83C00200
:1002C300C0031208F1AC82AD83D003D0028C028D3F
:1002D30003E4F54F754E0A8A828B83C002C0031272
:1002E300088FAC82AD83D003D00274302CFCE43D84
:1002F300FD8C4BE4F54F754E0A8A828B83C002C096
:10030300031208F1AC82AD83D003D0028C028D03BB
:10031300E4F54F754E0A8A828B83C002C00312082C
:10032300F1AC82AD83D003D00274302CFCE43DFDEC
:100333008C4C7C007D00EC2448F88606BE3010C34C
:10034300EC9405ED940050070CBC00EA0D80E78C9B
:10035300028D03BC050BBD0008EC24FFFAED34FF4E
:10036300FB8A048B050ABA00010BEC2448F8868249
:10037300C002C0031200A7D003D002C3EA9405EB66
:10038300940040DD2230980912009EAA828A3780A9
:10039300037537FF22120388AA82AB83BA1310BBFB
:1003A300000D120388AA82AB83BA11F6BB00F322B5
:1003B300E537B4654CD2B3D2B4C2B5C2B6C2B71234
:1003C3000081C2B390006412004FE4F531F530C3ED
:1003D300E5309401E53164809480501AC2A79000FF
:1003E3000A12004FD2A790000A12004F0530E4B55D
:1003F30030DD053180D9D2B390006412004F120171
:10040300AF22E537B477028003020493D2B3C2B4B8
:10041300D2B5D2B6D2B7D2A7120081E536B4FF0265
:10042300C2B390006412004FE4F53BF53AE4F531B2
:10043300F530AA30AB31C3EA953CEB953D50467598
:1004430082111200A7853038853139853890AA3951
:100453007B004302808AA012008112009EAA828A36
:10046300807582131200A7AA807B00EA253AF53A29
:10047300EB353BF53B12003830B2FD0530E4B530C7
:1004830002053180ADD2B390006412004F1201AF68
:1004930022E537B472028003020513E4F53BF53A13
:1004A300D2B3D2A7C2B4D2B5D2B6D2B77534317AE9
:1004B300007B00C3EA953CEB953D50518A388B395C
:1004C300853890AC397D004304808CA0C2B5C0024E
:1004D300C003120081D003D0027580FFAC807D0081
:1004E300EC253AF53AED353BF53B858082C002C0F9
:1004F300031201E3D003D002D2B5C002C00312033A
:1005030098D003D0020ABA00010B0204B61201AF5D
:1005130022E580B4FF02800B7534300540E4B5401A
:1005230002054122E537B46C40C2B3D2A7D2B7D299
:10053300B6D2B5D2B490006412004F1200389000C6
:100543000512004FC2B7C2B61200811200389000E4
:100553000512004FC2B5D2B6C2B7120081120038DD
:1005630090000512004F1201AF22E537B463267ADB
:10057300337B087C028A828B838CF01200B1E53ACC
:10058300F4FAE53BF4FB74012AF582E43BF58312AC
:1005930002041201AF22D2A7D2B3C2B4D2B5C2B7FA
:1005A300C2B6E4F5397538317590317A007B004372
:1005B30002808AA0C2B51200817580FF858035D282
:1005C300B50538E4B538020539853890AA397B007A
:1005D3004302808AA0C2B51200817580FF858036F0
:1005E30022120599E535B45102802AE535B4520249
:1005F3008033E535B45502803CE535B46102801D96
:10060300E535B462028026E535B46502802FE53511
:10061300B4FF378030753E00753F10802D753E0066
:10062300753F108025753E00753F20801D753E0087
:10063300753F208015753E00753F50800D753E0057
:10064300753F508005E4F53FF53EE4F53BF53AE4AC
:10065300F541F540D2A7D2B3C2B4D2B7D2B6D2B520
:100663007534317A007B00C3EA953EEB953F5042E7
:100673008A388B39853890AC397D004304808CA04F
:10068300C2B5C002C003120081D003D0027580FF3F
:10069300AC807D00EC253AF53AED353BF53BC002E5
:1006A300C003120514D003D002D2B50ABA00010B5D
:1006B30080B522E537B4730E120111AA82AB838A87
:1006C3003C8B3D1201AF22E537B46702800302077A
:1006D3006F1205E4E535B4FF0302075D7A407B083A
:1006E3007C028A828B838CF01200B18535821201E1
:1006F300E3E536B4FF0F7A4D7B087C028A828B8355
:100703008CF01200B1E536B4050F7A527B087C02F7
:100713008A828B838CF01200B17A567B087C028A22
:10072300828B838CF01200B1854082854183120253
:100733001F7A637B087C028A828B838CF01200B160
:100743007A6A7B087C028A828B838CF01200B185E3
:100753003C82853D8312021F800F7A7C7B087C02DA
:100763008A828B838CF01200B11201AF22E537B479
:10077300702A1205E48535821201E375822C12007A
:10078300A785408285418312021F75822C1200A720
:10079300853C82853D8312021F1201AF22E4F531AD
:1007A300F530E4F53DF53C759852758920758DFD5E
:1007B300D28E12008F7AEB7B077C028A828B838C2A
:1007C300F01200B11200E912019F1200F91206B6ED
:1007D3001203B312040512049412052712056D12B5
:1007E30006CA12077080E0220A0D20456173792D35
:1007F300446F776E6C6F616465722056322E3020C1
:10080300666F722041544D454C2038394335312FA2
:1008130035322F3535202873646363207665727310
:10082300696F6E29000A0D203E000A0D206F6B00D0
:100833000A0D2043484B53554D203D20000A0D20FF
:10084300666F756E6420383943002D313256002DA2
:100853003556000A0D206E6F6E626C616E6B200060
:10086300206279746573000A0D20627974657320C0
:10087300636F756E74657220000A0D204E6F7420CD
:10088300666F756E6420383943787800AA82AB832B
:100893007C007D007E10EB235401FFEBCA25E0CAE8
:1008A30033FBEDCC25E0CC33FDEF6003430401C300
:1008B300EC954EED954F400CC3EC954EFCED954FEA
:1008C300FD430201DED08A828B8322AA83AB828B13
:1008D300F0E54EA4F8A9F08AF0E54EA429F98BF0CF
:1008E300E54FA429F5838882222275820022AA82F9
:1008F300AB837C007D00E54F235401FE7028AE4E90
:10090300E54FCE25E0CE33FF8E4E8F4FC3EA9EEBED
:100913009F500E8E4EEFC313C54E13C54EF54F8039
:10092300050D8D0480D0C3EA954EEB954F4009C366
:10093300EA954EFAEB954FFBE54FC313C54E13C52E
:100943004EF54F8C051CED70DD8A828B8322C8C067
:10095300E0E5F0600D14600F14600F14601074FF75
:10096300800FA882E6800AE08007E4938003A882D0
:06097300E2F8D0E0C8220A
:00000001FF
